:10000000CFC3000005C4000003C4000001C4000009
:10001000FFC30000FDC30000FBC30000F9C30000E4
:10002000F7C30000F5C300000C94C12D0C94A92E59
:100030000C94762DEDC30000EBC30000E9C3000073
:10004000E7C30000E5C30000E3C30000E1C3000014
:10005000DFC300000C949D2DDBC30000D9C300005A
:10006000D7C30000D5C30000D3C30000D1C3000034
:10007000CFC30000CDC30000CBC30000C9C3000044
:10008000C7C30000C5C30000C3C30000C1C3000054
:10009000BFC30000BDC30000BBC30000B9C3000064
:1000A000B7C30000B5C30000B3C3000005010902D7
:1000B000A10185020901A1000509190129081500FE
:1000C0002501950875018102050109300931158165
:1000D000257F95027508810609381581257F9501D0
:1000E00075088106050C0A38021581257F95017572
:1000F000088106C0C005010980A101850319012AF4
:10010000B700150126B700950175108100C0050CD8
:100110000901A101850419012AA002150126A002E6
:10012000950175108100C005010906A1018506052C
:100130000719E029E71500250195087501810205D9
:1001400007190029EF1500250195F07501810205B9
:10015000081901290595057501910295017503910D
:1001600001C00660FF0961A1010962150026FF00B8
:100170009520750881020963150026FF00952075FA
:10018000089102C005010906A101050719E029E748
:1001900015002501950875018102950175088101F9
:1001A0000507190029FF150026FF0095067508812F
:1001B000000508190129051500250195057501910E
:1001C00002950175039101C00000000000000000CD
:1001D000000000000000000000000000000000001F
:1001E0000000000000000000000000007E0F00D4AE
:1001F000FFFFFFC7000000780000000000000000C3
:100200002A2B280000000000000000000000000071
:1002100000000029000000002C1E3420212224347C
:100220002627252E362D3738271E1F20212223244E
:1002300025263333362E37381F0405060708090AEA
:100240000B0C0D0E0F101112131415161718191A86
:100250001B1C1D2F3130232D350405060708090A04
:100260000B0C0D0E0F101112131415161718191A66
:100270001B1C1D2F3130354C09025B00030100A00F
:10028000FA09040000010301010009211101000124
:10029000224400070581030800010904010002034C
:1002A000000000092111010001222200070582033C
:1002B00020000107050303200001090402000103D7
:1002C00000000009211101000122B6000705840386
:1002D00020000112010002000000085A442113000E
:1002E00002010203011C037600690061006C003A00
:1002F00000660036003400630032006200330063A1
:10030000000000180344005A003600300052004735
:100310000042005F0057004B004C0000000E0344F9
:10032000005A00540045004300480000000403093F
:1003300004167C1E001F0020002100220023002440
:10034000002500260027002D002E0031002B001470
:10035000001A000800150017001C0018000C0012FD
:100360000013002F0030002A003921040016000776
:100370000009000A000B000D000E000F00330034CE
:10038000004C002800E1001D001B000600190005BC
:100390000011001000360037003800E50000002290
:1003A00052E000E300E200000000002C000000002A
:1003B0000000000000E60021520000E40035003A91
:1003C000003B003C003D003E003F00400041004239
:1003D00000430044004500010001000100520001FB
:1003E0000001000100B20001004900010046004781
:1003F000004800007C0100500051004F0001000146
:100400000001000100010001004A004B0001000151
:1004100000AC00AA00A900A80001000100137001AF
:100420000001004D004E00AB000000010001000182
:1004300000010000000000010000000000000000BA
:1004400000010001000000010001003A003B003CF7
:10045000003D003E003F0040004100420043004498
:100460000045004C00010020780100237824782505
:10047000782678277828782178010001000100008B
:100480007C010001000100010001000100010001E8
:100490000029782A78010001000100010001000113
:1004A0000001000100010001000100010001000144
:1004B0000001000100000001000100010001000036
:1004C0000000000100000000000000000001000129
:1004D000000000010001000100BF03231577150093
:1004E0000002000200BB0323157715000003000182
:1004F00000C00323157715000004000200A50323A4
:10050000157715D10705000100C1032315771500E4
:100510000006000200A7032315771500000700025C
:1005200000BD0323157715000009000200A903236D
:10053000157715DA070A000200AB0323157715DAE1
:10054000070B000200AD0323157715DA070C000234
:1005500000AF0323157715DA070D000200B103235E
:10056000157715DA070E000200B30323157715DAA5
:10057000070F000200B50323157715DA07100002F4
:1005800000B70323157715DA0711000200B903231A
:10059000157715DA0712000200C30323157715003B
:1005A0000013000200C50323157715000014000195
:1005B00000C703231577150000150000000000FF99
:1005C00007910F000016000100C2033A158E1500B6
:1005D0000017000101C2033A158E15000018000132
:1005E00002C2033A158E15000019000200C9032348
:1005F00015771500001A000103C2033A158E150085
:10060000001B000200CB03231577150000FD377A8D
:10061000585A000004E6D6B4460200210116000034
:1006200000742FE5A3E00316010A5D003D8889A64A
:1006300054750A36E182AEFA7A1AA6FCA2ED495444
:10064000B48A5E7177BBD0558E03A589CA55AFBCFD
:10065000CD23D6525448597C1B6297F0254409ADEE
:1006600002D29F1CB70E998B5A308891F64E4CF0EF
:100670009499716186D0A3D0DB48AA9CF94B5DAFF9
:10068000B9B8DCC5A5CC3369DAA48CA29C358C9AA8
:1006900063CF78EE5415F6585978F312946A81C9ED
:1006A000EAA89DC2693F84BA0DE4C878CAB8F66169
:1006B0000C359CA646EA4563E8331B1F09CB9DA970
:1006C0000C04A465070B35378FF18975267C786F8C
:1006D0006B331462061F986FC6729EBF9DBA559306
:1006E000E72C051FB8614CE2D6D270FABFB5A6DC84
:1006F000ACE83C2138D70BEC8545AB3E0BE1AEF2C4
:10070000264853882D3BBF71ECB4664DC6D557A61D
:10071000C6BE6D395CDBE423C2A9421F895C6D1F34
:100720002FDC65FEC5EE2164A4AF0395458611E478
:1007300089D4497F1BDC0000006CE32DFF5B0A714C
:10074000DD0001A60297060000E1D0CA52B1C467DD
:10075000FB020000000004595A4C4C4C4C4C4C4CD1
:10076000525252525252524C4C4C4C4C4C4C525293
:1007700052525252524C4C4C4C4C4C4C5252525283
:100780005252524C4C4C4C4C4C4C525252525200C5
:10079000524C4C4C00002A00000000525200520003
:1007A00011241FBECFEFDAE0DEBFCDBF04B603FEDB
:1007B00018C08091D2039091D303A091D403B0913B
:1007C000D5038730904BA740B04B59F41092D20319
:1007D0001092D3031092D4031092D503E0E0F8E313
:1007E000099511E0A0E0B1E0E6EBF0E602C005906B
:1007F0000D92A43BB107D9F723E0A4EBB1E001C00F
:100800001D92A23DB207E1F70E94AC260C94E62FA0
:10081000F7CB9C01FB019A9581159F4120F5832F11
:100820008170B32FB270AA27732F74706627532F6D
:100830005870442734FF0DC08295807FAB2B09F0A0
:100840008062672B09F08064452B09F08068099568
:100850000895AB2B09F08260672B09F08460452B6B
:10086000B1F38860F4CF80E0F2CF282F92959F708B
:10087000963099F060F4925F9F70923030F4203F90
:10088000B1F038F481E0283E38F080E008959A5FB6
:10089000F3CF81E0243FC9F7089591E0813F09F04B
:1008A00090E081E0283E08F080E0892B089581E007
:1008B000089580935903089580935A03089521E081
:1008C00030E001C0220F8A95EAF780915A03822B0B
:1008D000F3CF21E030E0A90102C0440F551F8A95F3
:1008E000E2F7CA01809590915A038923E5CF292F19
:1008F000953090F58E3080F590E03EE0239F800D9E
:10090000911D1124282F277041E001C0440F2A9522
:10091000EAF723E0969587952A95E1F7FC01EE0F1B
:10092000FF1FE80FF91FEC56FD4F20E030E070E0AC
:100930005191DF01CB01022E02C0969587950A9452
:10094000E2F7817081958527842385278E932F5F19
:100950003F4F2330310561F70895292F953078F501
:100960008E3068F590E03EE0239F800D911D1124AC
:10097000682F677023E0969587952A95E1F7FC012B
:10098000EE0FFF1FE80FF91FEC56FD4F40E050E05F
:1009900080E0219130E0062E02C0369527950A941A
:1009A000E2F721703327042E01C0220F0A94EAF7E0
:1009B000822B4F5F5F4F4330510559F7089580E018
:1009C000089590915A0321E030E0F90101C0EE0F43
:1009D0008A95EAF7D90102C0AA0FBB1F6A95E2F710
:1009E000EA2B01C0220F4A95EAF7892F8E23E813DC
:1009F00003C0892F822B60CF2095822F8923FBCFC4
:100A00008091930290E020E0022E001C000828173D
:100A100009060CF008952F5FF7CFFC01DB018481FC
:100A2000813041F514968C911497813019F591819C
:100A30008EE0E081F0E0899FE00DF11D1124E75A7E
:100A4000F84F94919A32B1F011962C911197EC9144
:100A5000F0E0829FE00DF11D1124E75AF84FE49178
:100A600081E09E1301C080E091E0EA3209F090E05D
:100A7000892B089581E008959C0180915B038D7915
:100A8000811119C0211540E5340780F4211580E259
:100A90003807C0F42333310511F1D0F481E02E3151
:100AA000310590F42430310530F00895C901965590
:100AB0008115914010F080E00895C901805F96454E
:100AC0000797C8F33327E6CF2C323105A1F70895F5
:100AD0002653310981E02330310538F3ECCF81E032
:100AE00008958091650390916403981301C008955F
:100AF0008F5F8770FACF90915F03809589238093F1
:100B00005F03282F2770211110C0891771F0909171
:100B1000CE0392FF0AC0869586958695DADE1092FE
:100B20005F031092610310926003089590915B033C
:100B3000982B90935B030895982F909580915B0379
:100B4000892380935B03089580915703811531F0C9
:100B50001092570310925603109255030895803E49
:100B60009105D9F1C8F48133910509F482C048F4A4
:100B70008932910509F472C08A32910509F480C066
:100B8000089589339105E9F082389105D1F08533D4
:100B9000910509F45EC00895843E9105D9F148F4A9
:100BA000823E910539F1833E910549F181EE90E055
:100BB0000895863E9105C9F1873E910509F43EC02E
:100BC00008952091CD032370211164C02091CE039C
:100BD00023FF14C089E290E008952091CD0320FD09
:100BE00045C03091CE0330FF09C024FD24C083EE00
:100BF00090E008952091CD0322FDF7CF0895209134
:100C0000CD0322FD44C03091CE0330FD43C024FF0C
:100C1000F5CF11C02091CE0321FFF0CF8091CD03FD
:100C200084FD09C087EE90E008952091CD0323FF55
:100C3000E5CF24FFF7CF80E090E008952091CD0329
:100C400023FD2BC03091CE0331FFE1CF84EE90E045
:100C500008952091CD0325FFD1CFBCCF2091CD03A6
:100C600025FD1EC02091CE0323FFC8CF89E390E06D
:100C700008952091CD0326FFC1CF8AE290E0089528
:100C80002091CD0326FFBACF81E390E0089582EE54
:100C900090E0089580EE90E0089586EE90E008954B
:100CA00085E390E008959091CD0392FF10C041E05C
:100CB000282F2471243009F040E031E0282F2871DA
:100CC000283009F030E0431711F02CE0822793FF21
:100CD00010C041E0282F2471243109F040E031E0B8
:100CE000282F2871283109F030E0431711F02CE04B
:100CF00082273091CE0330FF10C051E0282F2171A0
:100D0000213009F050E041E0282F2871283009F007
:100D100040E0541711F029E0822731FF10C041E074
:100D2000282F2171213109F040E031E0282F28716E
:100D3000283109F030E0431711F029E0822794FDB3
:100D4000877E08951F93CF93DF9309DFEC01811510
:100D500022E5920708F052C0811540E5940708F09B
:100D6000CDC0803E910520F58D3C910508F0A1C0D5
:100D7000883A910570F4853A910508F097C0813062
:100D80009105B9F10497813A910598F1C0E0D0E05E
:100D900030C0885A91094B97C8F7C85AD0E0CC0F99
:100DA000DD1FC95BDE4F0990D881C02DD46421C0FE
:100DB000811550E49507B0F4C11580E2D80708F01A
:100DC000B3C0C83ED105A8F0CE019A9581159F41C8
:100DD000E8F68D2F68DF182FCE019927C0DEEC01D1
:100DE000D12B07C09927BBDECC27DF70C82BD92BAE
:100DF000D06ACE01DF91CF911F910895803842E5EE
:100E00009407C8F5803652E5950708F05BC0C034FA
:100E100082E5D807D0F4C03292E5D90708F04BC07C
:100E20008C2F8695869520E2829FC0011124C37085
:100E300021E030E0A90102C0440F551FCA95E2F736
:100E4000EA01C82BD92BDD68D4CF8C2F86958695E7
:100E5000877050E2859FC0011124C37021E030E00B
:100E6000A90102C0440F551FCA95E2F7EA01C82B39
:100E7000D92BDC68BECF803C52E5950758F48F71C2
:100E8000C03AD245A0F590E0982F8827EC01C46FB6
:100E9000D06AAFCF805C9245809708F077CFDC2F87
:100EA000CC27CC27DF71C06FD06AA3CFA497D064C2
:100EB000A0CFD0659ECFCF71D0E0DC2FCC27C16F03
:100EC000D06A97CF86958695877020E2829FC00171
:100ED0001124C37021E030E0A90102C0440F551F66
:100EE000CA95E2F7EA01C82BD92BDA6882CFDBDE9C
:100EF000C82FD0E0DC2FCC27D0627BCF8F71D3DE20
:100F000093E0CC0FDD1F9A95E1F7CC27DF70282FF7
:100F100030E084FF05C050E1859F90011124332704
:100F2000C22BD32BD06965CF8D2F8F71BCDE182FCC
:100F3000CE01992714DEEC01D12BDECF80E008959D
:100F4000F894E82FE295EF70F0E041A18F7021E076
:100F500030E0B90102C0660F771F8A95E2F7CB0136
:100F6000962F9095942391A392A1892B82A3789494
:100F70000895E4ECF2E080E090E064EC75E247EE86
:100F800055E229E536E277836683518740873387C8
:100F9000228797878687019670968830910599F702
:100FA00008958091A5039091A603909311018093D9
:100FB00010010895E5EAF3E0848195812AE030E0AC
:100FC000B9010E94F42E609314018681809315016B
:100FD00082858093030184858093020186859785AD
:100FE000B9010E94F42E609312018089809313014D
:100FF0008289809301018489809300010895EF9292
:10100000FF920F931F93CF93DF93FB018FEF9FEF1F
:101010004430510508F45FC04091CD0341FB88275F
:1010200080F990E0880F991F42FB002700F910E03B
:10103000000F111F000F111F802B912B40FBEE247E
:10104000E0F8F12C8E299F2943FB222720F9C22F9B
:1010500050E0D52F53E0CC0FDD1F5A95E1F78C2BD4
:101060009D2B44FB222720F950E1259F900111245C
:10107000822B932B45FB222720F950E2259F9001DC
:101080001124822B932B46FB222720F950E4259F25
:1010900090011124822B932B47FB222720F940E853
:1010A000249F90011124822B932B2091CE03322F69
:1010B0003170932B26952170B22FBB0FA0E08A2BA5
:1010C0009B2B092E000CAA0BBB0B80839183A28360
:1010D000B38380E090E0CDB7DEB7E6E00C94502F0C
:1010E000AC0123E0969587952A95E1F78E719927B3
:1010F000FC01E250FE4F0190F081E02D4F7055272A
:1011000021E030E002C0220F331F4A95E2F761155B
:1011100041F0E22BF32B82509E4FDC01ED93FC93C8
:10112000089520953095E223F323F5CF282F35EB52
:101130002303C001112497FF04C080589109892F0F
:10114000089580589F4FFBCF8091B1026091AD030D
:101150007091AE0380FF14C020910301269FC0014F
:10116000279F900D1124BC0176956795769567951C
:1011700060387105F0F561157105E9F1862F089564
:1011800081FF0BC020910301269FC001279F900D76
:101190001124BC0176956795EBCF82FF09C0809141
:1011A00003019B01829FB001839F700D1124E0CF4A
:1011B0008091B0028115E1F290910201209103012A
:1011C000891738F0CB01289FB001299F700D112499
:1011D000CFCF289F90011124269FA001279F500D5B
:1011E000369F500D1124692F70E0CA010E94F42E21
:1011F000BFCF8FE7089581E008958091B10280FF0D
:101200000CC06091010170E07595679575956795C3
:101210006115710549F1862F089581FF06C060911F
:10122000010170E075956795F3CF6091010182FD32
:101230000BC09091AF029115A1F0609100018091D7
:101240000101961738F0682F70E06038710500F3DF
:101250008FE70895899FC001112470E00E94082F34
:10126000F4CF61E070E0D7CF81E00895FA013097C4
:1012700009F009950895E0917902F0917A0230978A
:1012800039F00190F081E02D309711F00995089523
:1012900080E00895A3E0B0E0E0E5F9E00C94382F99
:1012A0009C018091FC019091FD0182179307B1F0A0
:1012B0003093FD012093FC01E0917902F0917A02D4
:1012C000309761F00084F185E02D309739F083E0AC
:1012D00089833B832A83CE01019609952396E2E018
:1012E0000C94542FA3E0B0E0E8E7F9E00C94382F19
:1012F0009C018091FA019091FB0182179307B1F054
:101300003093FB012093FA01E0917902F0917A0287
:10131000309761F00084F185E02D309739F084E05A
:1013200089833B832A83CE01019609952396E2E0C7
:101330000C94542F90911801913091F0A8EBB1E0EA
:10134000EFEF90E02D91821751F0EF3F19F421114A
:1013500001C0E92F9F5F9630A9F7EF3FC9F40895C8
:101360009091CD0397FFEACFE82FE695E695E695B5
:10137000803FA8F7F0E0E254FE4F877021E030E0B4
:1013800001C0220F8A95EAF78281822B8283089519
:101390000E2E000CFF0BEA54FE4FF8CF909118016F
:1013A000913021F49091CD0397FD0CC0E8EBF1E072
:1013B0009191891302C0DF011E9251E0EE3BF507C7
:1013C000B9F70895E82FE695E695E695803FC8F7CA
:1013D000F0E0E254FE4F877021E030E0A90102C046
:1013E000440F551F8A95E2F7CA018095928189239F
:1013F000828308958091170108952FB7F894809102
:10140000F6019091F701A091F801B091F9012FBF79
:1014100008958091A7039091A803892B89F0EDDFAF
:101420002091550330915603AC01421B530B9A0196
:1014300081E04091A7035091A8032417350708F4D1
:1014400080E00895CF93DF93C0915B0380915E03AA
:10145000C82B809157038115E1F08091A7039091EB
:10146000A803892B19F0D5DF81116EDBD0915703CA
:1014700080911801813021F48091CD0387FD0DC04A
:1014800086E028EB31E090E0815058F491115CDB6C
:10149000CD2B8C2FDF91CF9108958EE120EC31E0A0
:1014A000F2CFF90141919F01411571F39F5FECCF9C
:1014B000962F2091CE0322FF0EC0682F660F660F75
:1014C000660F692B60935F03FAD997DF90936103EE
:1014D000809360030895F3C990915703292F28231F
:1014E000211559F08095892380935703811531F098
:1014F00084DF8093550390935603089580E090E035
:10150000F8CFCF93C82F8091CE0382FF0BC080917C
:1015100057038C1739F071DF90935603809355036E
:10152000C0935703CF91089568DF2091B4023091A2
:10153000B502232B211521F080933F0290934002A6
:101540002091B6023091B702232B211521F0809310
:101550003D0290933E02E0917902F0917A02309739
:1015600059F00680F781E02D309731F082E08093CA
:10157000B20282EB92E009950895611509F441C029
:10158000E3E3E80FE33148F4F0E0E851F04D0C9468
:101590001B2FDADD81958093B502C6CFD5DDFBCF59
:1015A000D3DD81958093B402F8CFCEDDFBCF25DE6D
:1015B0008093B602F2CF21DE8195FACF1EDE8195AF
:1015C0008093B702EACF19DEFBCF815D990B21E052
:1015D00030E001C0220F8A95EAF78091B302822B96
:1015E0008093B302DACF8091B10281608093B1021F
:1015F000D4CF8091B1028260F9CF8091B102846032
:10160000F5CF4091B4028D3C59F48091B50287FF2B
:101610000DC01092B502411559F41092B00208C0E5
:101620008E3C81F48091B50218169CF3411581F02F
:101630008091B6029091B702892B8111AECF1092A2
:10164000AF02ABCF8F3C41F447FFF0CF1092B40212
:101650008091B5028115E0CF803D19F41416B4F3E2
:10166000E5CF9091B602893D29F41916FCF6109247
:10167000B602DCCF8A3D19F497FFD8CFF8CF90910E
:10168000B7028B3D29F497FFD1CF1092B702CECF8E
:101690008C3D19F41916CCF3C9CF9FE2980F9830FE
:1016A00090F4815D990B21E030E0B90102C0660F32
:1016B000771F8A95E2F7CB0180959091B302892339
:1016C0008093B302B3CF8D3D31F48091B1028E7F10
:1016D0008093B102ABCF8E3D21F48091B1028D7F1A
:1016E000F7CF8F3D09F0A2CF8091B1028B7FF0CF71
:1016F0002FB7F8946091F6017091F7018091F8018D
:101700009091F9012FBF0895FC019B018091EC019C
:101710009091ED018617970740F0672B29F480918F
:10172000E8008E778093E800C90140E0009741F41B
:10173000411106C08091E80082FF2FC080E008952B
:10174000209152022115A9F12530A9F12091E8003C
:1017500023FD2DC02091E80022FDECCF2091E80070
:1017600020FFE4CF3091F3002091F200009719F0B0
:101770002830310558F041E02830310509F040E0CB
:101780002091E8002E772093E800D0CF419140933C
:10179000F10001972F5F3F4FE9CF809152028115F1
:1017A00041F0853041F08091E80083FFC3CF81E0B4
:1017B000089582E0089583E008958091E60187FF0F
:1017C00013C08091E80082FF06C08091E8008B770B
:1017D0008093E8000895809152028111F2CF08951C
:1017E000809152028115D9F38091E80080FFF8CFF3
:1017F0008091E8008E77ECCF2091E4003091E500F5
:1018000095E6A9012091EC00822F817020FF06C08F
:101810008091E80080FF06C080E008952091E800F4
:1018200022FD1AC080915202811589F0853089F01D
:101830008091EB0085FD0FC02091E4003091E50020
:1018400042175307F9F29A95E1F684E0089582E091
:10185000089583E0089581E00895E8EDF0E0808147
:101860008E7F80831092E2001092DA001092E100E5
:10187000A0EEB0E08C9181608C9380818F77808323
:1018800019BCA7EDB0E08C918E7F8C9380818F7E08
:1018900080831092E5010895E0917902F0917A0237
:1018A000309739F00284F385E02D309711F060E233
:1018B00009950895982F9093E900891771F0709118
:1018C000EC002091ED005091F00021FD09C09F5FD8
:1018D000973089F78093E9000895762F242F50E000
:1018E0003091EB003E7F3093EB003091ED003D7F77
:1018F0003093ED003091EB0031603093EB0070934A
:10190000EC002093ED005093F0002091EE0027FDB5
:10191000DECF0895A0E0B0E0E0E9FCE00C94322FC7
:10192000C8EDD0E088818F7E8883E7EDF0E080818C
:101930008160808384E082BF81E08093E5018881BB
:101940008E7F888302EE10E0F80110821092DA0098
:1019500081EEC82ED12CF601108288818F77888382
:1019600088818068888388818F7D888319BC1092E4
:1019700052021092E401109231021092E30190EEB3
:10198000E92EF12CF70180818B7F80838881816033
:10199000888342E060E080E08DDFF60180818E7F09
:1019A0008083F8018081816080838081886080836A
:1019B000F70180818E7F8083888180618883CDB7A5
:1019C000DEB7E8E00C944E2FE0916503909164033C
:1019D00027E0E91302C080E00895AE2FB0E02E9F0B
:1019E000F0011124EA59FC4F3181361306C03081D1
:1019F000381303C03581341304C0FD013196E770FC
:101A0000E8CF81E008959C012115310509F408957E
:101A10008FE99FE00197F1F700C0000021503109E4
:101A2000F3CF81E08093E00080E28093D8001092B1
:101A3000C9008FE19EE40197F1F700C0000087E044
:101A400090EBDC018093D2039093D303A093D40353
:101A5000B093D50388E19CE00FB6F894A8958093E5
:101A600060000FBE90936000FFCF0F931F93CF9342
:101A7000DF938B01EA0190915202943051F58093EB
:101A8000E9008FEF9091E80095FD06C095ED9A95DD
:101A9000F1F700008A95B1F78091E80085FF19C041
:101AA000ABDE811111C08091E80085FD06C08091F8
:101AB000E8008E778093E800F3CFF80181918F01E1
:101AC0008093F100219779F78091E8008E778093D9
:101AD000E800DF91CF911F910F910895792F603227
:101AE00029F440E250E0682F82E0BFCF0895CF9301
:101AF000DF93D82FC92F48E050E0682F792F81E07D
:101B0000B4DF88E0ED2FFC2FAEEEB1E001900D9236
:101B10008A95E1F7DF91CF910895BC0140E250E052
:101B200084E0A3CFBC0146E050E084E09ECFBC013E
:101B300043E050E084E099CFFC016081718184E052
:101B400090E00C94CB2F9091CE0392FB222720F9AA
:101B5000281751F080FB92F99093CE038DEC93E01F
:101B6000EBDF82E00C947B0508951F93CF93DF9306
:101B7000962F122F632F8430D8F49530C8F44E304E
:101B8000B8F4C42FD0E0CC0FDD1F2CE1929FC00D24
:101B9000D11D11249CE8899FC00DD11D1124CE01B7
:101BA00089960E94B12F612FCE018A960E94B12F93
:101BB000DF91CF911F91089580911801813061F5D7
:101BC0008091CD0387FF28C03DDC8093BF0140E2B8
:101BD00050E069E572E08EEB91E00E94682F892B5E
:101BE000D1F080E2EEEBF1E0A9E5B2E001900D92D8
:101BF0008A95E1F7E0917902F0917A02309759F0F5
:101C00000480F581E02D309731F086E08093BE01AD
:101C10008EEB91E00995089515DC8093B60148E0BC
:101C200050E06BE772E086EB91E00E94682F892B11
:101C300091F388E0E6EBF1E0ABE7B2E001900D92C2
:101C40008A95E1F7E0917902F0917A02309719F3E1
:101C50000280F381E02D3097F1F286EB91E0DACF4C
:101C6000811519F00E949605A7CF0895811531F0CE
:101C700090915E03892B80935E039ECF089581151A
:101C800019F00E949C0598CF0895811539F0809530
:101C900090915E03892380935E038ECF0895CF9346
:101CA000C82F8115C1F08CEF8C0F813A80F580919F
:101CB0001801813021F48091CD0387FD0EC0E8EB3F
:101CC000F1E08191C817F9F021E0EE3BF207C9F786
:101CD0008C2F30DB71DFCF910895EC2FE695E695E0
:101CE000E695F0E0E254FE4F828190E04C2F477081
:101CF00021E030E002C0220F331F4A95E2F7822331
:101D00009323892B29F38C2F49DB56DFE1CF80E227
:101D10008C0F883048F4C77081E001C0880FCA95E5
:101D2000EAF70E949605D6CF8BE58C0F833030F40E
:101D30002C2F2452330BC901ADDACDCFE8E5EC0FDF
:101D4000EB3148F4F0E0EE0FFF1FE358FE4F8081C7
:101D50009181C8DAC0CF83E38C0F833108F0BBCF09
:101D600061E08C2F0ADCB7CFCF93DF93EC01805E6C
:101D70009109089720F066E37EE0209711F460E374
:101D80007EE0CE010E9409048C2F89DFDF91CF9184
:101D90000895611529F020915E03226020935E036F
:101DA0009C0130522115304308F49927DDCF81156D
:101DB00041F19CEF980F913A10F4F0DAFDCE90E2E9
:101DC000980F983050F4877091E001C0990F8A9570
:101DD000EAF7892F0E949C05F1CF9BE5980F93307D
:101DE00018F480E090E056CA98E5980F9B3118F4FB
:101DF00080E090E077CA93E3980F933110F460E0AD
:101E0000BCCB0895CF93DF93EC01D1DFCE01805E90
:101E10009109089720F065E47EE0209711F46FE3C4
:101E20007EE0CE010E940904DF91CF9108951F93B7
:101E3000CF93DF93182FEB0132DF209731F4812FFE
:101E4000B6DFDF91CF911F9108958FE99FE0019751
:101E5000F1F700C000002197F0CF6091C5037091A9
:101E6000C603893321F06091C3037091C403DFCFAF
:101E700010925B0380911801813011F58091CD03A0
:101E800087FF1EC0E0ECF1E08EE1DF011D928A9534
:101E9000E9F780E090E0FED980E090E023DA10924C
:101EA0005E038ADE86E0E2EBF2E0DF011D928A95B6
:101EB000E9F71092B0021092AF021092B10234CB47
:101EC000E8EBF1E086E0E1CFD3DF2FEF84E39CE0A5
:101ED000215080409040E1F700C0000088E19CE084
:101EE0000FB6F894A895809360000FBE90936000A1
:101EF000FFCFCF93DF93D82FC92F209193022830A3
:101F000010F0B6DF20E0E22FF0E0EE0FFF1FED57FC
:101F1000FD4FD083C1832F5F20939302DF91CF9138
:101F20000895CF93DF93FB018FEF9FEF443051056E
:101F300088F0D081C1819CDFD093CD03C3708091A4
:101F4000CE038C7FC82BC093CE038DEC93E0F4DDE1
:101F500080E090E0DF91CF910895AAE2B0E0E3EB5A
:101F6000FFE00C94372F86EE91E0FC010196209162
:101F7000F100208321E08E3E9207B9F78091E701BE
:101F8000893009F457C0C8F4823009F4B2C08330F4
:101F900009F482C0813081F18091E80083FFE6C0BE
:101FA0008091E6019091E7019A3008F0DFC0E92FB7
:101FB000F0E0E550F04D0C941B2F8A3009F489C0F5
:101FC0008B3051F78091E601813231F78091EA013F
:101FD0009091EB01892B01F78091E800877F809336
:101FE000E800EBDB81E09091E801911101C080E015
:101FF000809318013DDFD0CF8091E601813A61F6F0
:102000008091E800877F8093E8008091EA019091B9
:10201000EB01892B59F060E080E090E070E074DB28
:102020008091E8008B778093E800B6CF68E08EEE71
:1020300091E0F4CF8091E601813209F0ADCF80913B
:10204000EA019091EB018D7F892B09F0A5CF80915A
:10205000E800877F8093E8008091E80082FF17C046
:102060009091F3008091F200029731F48091F10099
:10207000813011F0863021F48091F10080931701B6
:102080008091E8008B778093E80097DB85CF809183
:1020900052028111E1CF80CF8091E601813A09F0AF
:1020A0007BCF8091EA019091EB01892B09F074CFED
:1020B0008091E800877F8093E8008091E80080FFAE
:1020C000FCCF809118018093F1008091E8008E7719
:1020D000DACF8091E601813209F05ECF8091E8008D
:1020E000877F8093E80069DB8091E9018093160186
:1020F00053CF8091E601813A09F04ECF8091E800FC
:10210000877F8093E8008091E80080FFFCCF80917A
:102110001601D9CF803889F0823841F58091EA01E3
:102120008F70873018F58093E9008091EB0085FB74
:10213000882780F91092E90006C080913102880F4B
:102140009091E301892B9091E800977F9093E800AC
:102150008093F1001092F1008091E8008E7723C007
:10216000811116C08091E801813009F18091E80069
:1021700083FF0AC08091E800877F8093E800809108
:10218000EB0080628093EB00AA96E3E00C94532F5F
:10219000823061F78091E801811581F01092E900A9
:1021A0008091E800877F8093E80007DBDFCF81E044
:1021B000933009F080E080933102F0CF8091EA0102
:1021C0008F702FEF280F263088F68093E90020913A
:1021D000EB0020FFE3CF933031F48091EB0080627D
:1021E0008093EB00DBCF9091EB0090619093EB003C
:1021F00021E030E0A90102C0440F551F8A95E2F7A3
:102200004093EA001092EA008091EB008860E8CFEA
:102210008111ACCF1091E8011F778091E3008078A5
:10222000812B8093E3008091E800877F8093E80012
:10223000C4DA8091E80080FFFCCF8091E3008068E1
:102240008093E30083E0111101C082E08093520289
:102250008DCF8058823008F089CF8091E80190912D
:10226000E9018C3D53E0950791F583E08A838AE28A
:1022700089834FB7F894DE01139620E03EE051E2E7
:10228000E32FF0E050935700849120FF03C0829524
:102290008F703F5F8F708A30C0F0895C90E08D93C3
:1022A0009D932F5F243161F74FBF8091E800877FB6
:1022B0008093E8006AE270E0CE01019625DA809111
:1022C000E8008B778093E80051CF805DE7CF292F1E
:1022D00033272330310509F44EC078F5213031051C
:1022E00009F488C08BE590E0E8E7F2E022303105A0
:1022F00009F03CCF2091E800277F2093E80020914F
:10230000EC013091ED018217930708F49C0140E045
:102310002115310509F073C0411171C08091E800A9
:1023200082FDCDCF80915202811549F2853039F27C
:102330008091E80083FFF2CFC2CF8091EA019091B3
:10234000EB012132310509F446C02232310509F092
:102350000DCF8330910508F009CFFC01EE0FFF1F70
:10236000E85DFE4F0190F081E02D8B5D9E4FDC011A
:102370008C9190E010C09C013327823021F12330F2
:10238000310568F4232BB9F4EDE2F3E0E4918E2FEC
:1023900090E0EDE2F3E0009709F4E8CEABCF233014
:1023A000310509F0E3CEE5EEF2E0E4918E2F90E006
:1023B000E5EEF2E0F0CFEDE1F3E0E4918E2F90E076
:1023C000EDE1F3E0E8CFE3E0F3E0E4918E2F90E07D
:1023D000E3E0F3E0E0CF8330910508F0C7CEFC01E5
:1023E000EE0FFF1FE25DFE4F0190F081E02D89E0CE
:1023F00090E080CF82E190E0E3EDF2E07BCF80914E
:102400005202811509F45BCF853009F458CF8091D1
:10241000E80083FD54CF8091E80082FD7FCF80915A
:10242000E80080FF75CF9091F3008091F2002115B4
:10243000310519F08830910550F041E0089709F016
:1024400040E08091E8008E778093E80061CF44916E
:102450004093F1003196215031090196E8CF803840
:1024600009F084CE8091E800877F8093E800809116
:10247000E4018093F10070CE811178CE1091E801D3
:10248000123008F073CE8091E800877F8093E800D7
:102490001093E40192D91115D9F084E0809352028F
:1024A00042E061EC81E006DA42E261EC84E002DACB
:1024B00042E261EC82E0FED942E260EC83E0FAD9CC
:1024C00080915202843051F482E0809319014ECE03
:1024D0008091E30087FDE1CF81E0E0CF81E0F5CF9F
:1024E00080911A01877F80931A0190915E039D7FEE
:1024F00090935E0384FF06C08F7E80931A0182E072
:102500000E94960580911A0185FF06C08F7D8093F9
:102510001A0180E20E9496054FCBCF92DF92FF9284
:102520000F931F93CF93DF93EC018B01F42E8091D7
:102530001A0182FF61C0C0904A03D0904B03CC16B1
:10254000DD0619F0209709F057C080911A018B7FA2
:1025500080931A01C1E081FD10C0809148039091E1
:1025600049039801281B390BC1E08091100190911B
:1025700011012817390708F4C0E080911A01C0FB47
:1025800081F980931A016C2FC6010E947008809116
:102590005B0381FF08C080911A01806180931A015A
:1025A00082E00E949C0580915B0385FF08C08091BA
:1025B0001A01806280931A0180E20E949C056C2FB0
:1025C000C601E7DBF11431F08091C00385FF02C042
:1025D00086FF25C08091C3039091C40314DA8091D3
:1025E0004A0390914B039C0130522115304308F46B
:1025F000992708DC75DF0FC0CE01905281159043FA
:10260000B0F4CE019927FEDB80914A0390914B03F1
:10261000C817D90779F31093490300934803DF9152
:10262000CF911F910F91FF90DF90CF900895CE0131
:10263000EACFCF93DF93EC014A855B856E857F857A
:102640000E9436099B81909580915E038923809337
:102650005E038C810E949C05AFDA86E0FE01119238
:102660008A95E9F7DF91CF910895CF93DF93EC013D
:102670008D8181FD13C082608D8380915E039B817B
:10268000892B80935E038C810E94960595DA48859C
:1026900059856E857F85CE010E94360910924503CB
:1026A000109244038D8180FD02C0CE01C2DFDF9114
:1026B000CF9108950F931F93CF93DF9305EA13E013
:1026C000C9E5D2E0CE010E94952FF80161918F01FA
:1026D000681719F0CE010E94B12F2196C138F2E09F
:1026E000DF0781F7DF91CF911F910F9108950F932D
:1026F0001F93CF93DF9305EA13E0C9E5D2E0CE0143
:102700000E94952FF80181938F012196C138F2E044
:10271000DF07A9F7CFEDD4E0FE01859195910097F1
:1027200011F0FC0109952C96F6E0C731DF07A1F7FF
:10273000DF91CF911F910F910895E5EAF3E0128E9A
:10274000138E8FEA90E09183808325E0248F88E8C0
:1027500093E1938382838AE090E09583848344E1CC
:1027600050E05783468348E050E051874087938785
:1027700082876EE170E0758764879787868780E53A
:1027800090E0918B808B538B428B48E250E0558BCD
:10279000448B42E350E0578B468B48EC50E0518F1E
:1027A000408F158E55A344A3178E168E91A380A338
:1027B00022A317A216A27EDF5BDB1092CE0310923B
:1027C000CD0380E084608093CE038DEC93E0B4D998
:1027D0008ECF0F931F93CF93DF93843030F5653006
:1027E00020F54E3010F5C42FD0E0CC0FDD1F2CE1CA
:1027F000629FC00DD11D11243CE8839FC00DD11DE7
:102800001124CE0189960E94952F082F10E0102FD9
:102810000027CE018A960E94952F9801282BC90186
:10282000DF91CF911F910F91089580E090E0F8CF54
:10283000462F672F2091550230915602232B81F4A9
:10284000703F39F4403F61F48091530290915402FB
:102850000895753028F44E3018F4843008F4B9CF58
:1028600080E090E00895A0E0B0E0E9E3F4E10C94AA
:10287000332F7C0100915A0380915903082BC3E048
:10288000D0E010E0C8010C2E02C0959587950A94FF
:10289000E2F780FD09C02197A8F7D12C8D2DCDB787
:1028A000DEB7E7E00C944F2FDC2EB7018C2FC0DF92
:1028B0000E94A206019779F3F1CFCF93DF93D82F2F
:1028C000C92FD1DF6D2F7C2FB3DF0E94A206DF91CD
:1028D000CF910895FC018481811529F08081918137
:1028E000ECDF0C94350480E008951F93CF93DF93C1
:1028F000182FD92F611589F0411579F0B4DFC82F51
:10290000682F812F9D2F0E947704612F7D2F8C2FA0
:102910008FDFDF91CF911F9108950E94AD04C82FE2
:10292000F4CFFC01462F658180819181DECF382F65
:10293000292FCB01A32FB22F8F3221E09207A105BF
:10294000B10520F48F529D4F0C94952F80E008958F
:1029500085E290E00E94952F873A89F486E290E024
:102960000E94952F8A3859F487E290E00E94952FB3
:1029700091E0843409F090E0892F8170089580E01F
:10298000FCCFAAE0B0E0E7ECF4E10C942D2FA0908E
:102990005002B090510281E090E0909351028093F8
:1029A0005002812C912C10E0640100E019C021E05C
:1029B00030E0133021F0F701859195919C01472D6E
:1029C000602F812FD2D8739422E0E20EF11C3EE0FA
:1029D0007312EDCF0F5F8EE0C80ED11C053049F0A9
:1029E000C601880F991F9C012F5C3C4F7901712C07
:1029F000DECF1F5F36E4830E911C1430A9F69DDEF6
:102A00001A8219821C821B821E821D8218861F82D6
:102A100088EC90E09A87898701E812E04AE050E06C
:102A2000B801CE0101960E94CF2F065F1F4F013DD6
:102A300082E0180799F7B0925102A09250022A96AC
:102A4000EDE00C94492F9C01CB01BA01F9013296BB
:102A5000E4914E2F50E06E17710548F0F90134965D
:102A6000659175910E94752F80E090E008958FEF39
:102A70009FEF0895A4E0B0E0E0E4F5E10C94352F79
:102A80008B01FC013396F49019821A821B821C82FE
:102A9000452B31F48FEF9FEF2496E5E00C94512FF6
:102AA00044E050E0BE016F5F7F4FCDDF019691F3B0
:102AB00081E090E00F2C02C0880F991F0A94E2F782
:102AC000092E000CAA0BBB0B49815A816B817C81BA
:102AD00084239523A623B72321E0892B8A2B8B2BD4
:102AE00009F420E0F801208380E090E0D5CF9C013C
:102AF000CA01F9013296E4914E2F50E08E179105EC
:102B000050F0F9013496859195910E94752FD2DD90
:102B100080E090E008958FEF9FEF0895A4E0B0E08B
:102B2000E4E9F5E10C94312F7C016B01CA01F70156
:102B30003396B49019821A821B821C82892B31F43D
:102B40008FEF9FEF2496E9E00C944D2F44E050E086
:102B5000BE016F5F7F4FC70176DF019689F381E089
:102B600090E00B2C02C0880F991F0A94E2F7809521
:102B70009095092E000CAA0BBB0B49815A816B81E1
:102B80007C8184239523A623B723F6012081022F7D
:102B9000017010E00B2C02C0000F111F0A94E2F725
:102BA000012E000C220B330B802B912BA22BB32B6D
:102BB00089839A83AB83BC8344E050E0BE016F5F9E
:102BC0007F4FC70194DFBECFAAE0B0E0EAEEF5E1A7
:102BD0000C942C2FFE0131968AE0DF011D928A951C
:102BE000E9F794E3A92E91E0B92E8F013F01EE247D
:102BF000E394F12C37E4C32E31E0D32EF50181911B
:102C00005F018F3F09F444C0F894E82FE295EF701C
:102C1000F0E021A18F70A70102C0440F551F8A95D3
:102C2000E2F7CA01922F982B91A392A18095892354
:102C300082A3789400C0E9E3F1E021E030E0812C48
:102C4000912C41914F3F79F0A42FA295AF70A05ED7
:102C5000B0E08C9190E04F7002C0959587954A95B1
:102C6000E2F780FF3BC080E090E0882A992A220F9B
:102C7000331FCE16DF0629F7F50182918F3F11F041
:102C80000E94A00750EA5A95F1F7D8018D929C92C4
:102C90000E5F1F4FB9E3AB16B1E0BB0609F0AECF34
:102CA0004AE050E0B30186E292E00E94682F892B4F
:102CB000B9F08AE0F301A6E2B2E001900D928A95A4
:102CC000E1F781E08093E0010E94FD099093DF012C
:102CD0008093DE012A96EEE00C94482FC901C5CFFF
:102CE0008091E0018115B1F30091DE011091DF01C7
:102CF0000E94FD09801B910B039760F34AE050E0AE
:102D000066E272E086E492E00E94682F892B49F027
:102D10008AE0E6E2F2E0A6E4B2E001900D928A9544
:102D2000E1F71092E001D6CF282FCB01283070F4C4
:102D30004AE0249F90011124B9016F577D4F4AE06A
:102D400050E00E94852F80E090E008958FEF9FEF84
:102D50000895AAE0B0E0EFEAF6E10C94382F9C0168
:102D600097558115914068F4BE016F5F7F4F822FA8
:102D7000DBDF892B31F489859A852A96E2E00C9471
:102D8000542F8091BD039091BE03F7CFA0E0B0E037
:102D9000ECECF6E10C94332F162FD72FC42FD22E44
:102DA0008115A9F0409353030E94FD099093E2011D
:102DB0008093E101C77081E001C0880FCA95EAF7EE
:102DC0000E94300ECDB7DEB7E7E00C944F2F909104
:102DD0005303491336C0E090E101F090E2010E94F4
:102DE000FD099C012E193F097901812F9D2FB1DF2B
:102DF000E816F90630F5D0E2DD0DCD15A1F0C7706B
:102E000011E0812F01C0880FCA95EAF70E943F0E9A
:102E1000D83048F48D2D877001C0110F8A95EAF7DC
:102E2000812F0E94300E802F18D8D83058F62D2DC3
:102E3000277081E001C0880F2A95EAF70E943F0EB3
:102E4000C1CFC77081E001C0880FCA95EAF7F6CFFD
:102E5000A0E1B0E0EEE2F7E10C942A2FFE013196FA
:102E600080E1DF011D928A95E9F703E110E091ED21
:102E7000A92E92E0B92E2FE2422E55245394612CB4
:102E8000712C4F0173016201B1E14B1651046104D1
:102E900071041CF080E1C82ED12CA601B501C4013B
:102EA0000E94A22FAC0CBD1C0D2C000CEE08FF08DC
:102EB0004C185D086E087F080150104019F76096A5
:102EC000E0E10C94462F6FEF85E290E00E94B12F75
:102ED0006FEF86E290E00E94B12F6FEF87E290E003
:102EE0000E94B12F60E088E290E00E94B12F49DD9E
:102EF000AFDF67EA85E290E00E94B12F6AE886E2E0
:102F000090E00E94B12F64E487E290E00C94B12F2E
:102F1000A0E0B0E0EEE8F7E10C94312FEC018881FD
:102F20008115F1F0813009F042C08981813029F4A6
:102F30008A8123960E942D0FF2CF823029F48A8154
:102F400023960E944F0EEBCF833029F48A8123967B
:102F50000E94D70EE4CF843041F022968111DFCF5A
:102F6000CDB7DEB7E9E00C944D2F8A81239620E09F
:102F700030E09AE0682F6053770BAB016A3071053F
:102F800060F02115310551F3EFE9FFE03197F1F7DA
:102F900000C0000021503109F4CF929FB001939FEF
:102FA000700D11249A01260F371F8991E3CFE82F66
:102FB000F0E0E850FE4FB490282F269526952695F0
:102FC00030E0F901E851FE4FE4908770F12C082EB3
:102FD00002C0F594E7940A94E2F7E0FAEE24FF24A5
:102FE000E0F8F901E852FE4FC490D12C082E02C03F
:102FF000D594C7940A94E2F7C0FACC24DD24C0F833
:10300000F901E853FE4F049110E002C015950795B1
:103010008A95E2F701701127E114F10419F081EEAD
:103020000E944F0EC114D10419F086EE0E944F0E7B
:1030300060E070E08B2D0E94170FC114D10419F0CD
:1030400086EE0E94D70EE114F10419F081EE0E9481
:10305000D70E0115110519F08CE20E942D0F219653
:103060005ECFAAE0B0E0E7E3F8E10C942A2F7C0100
:10307000DC0114968C91811509F458C360E0C701F6
:1030800050DC9C01F7018681803170F4409165032A
:1030900090916403491333C09091A303911521F0DB
:1030A0009091A403903158F1D70115969C919111FC
:1030B00010C02115B0E53B0708F0ACC02115E0E2D7
:1030C0003E0708F0BCC0283E310590F4203E310593
:1030D000B0F43093B9022093B802D70112968D91C3
:1030E0009C91909363038093620310921B0107C02D
:1030F000C9019A9581159F4160F72111EACF61E0DE
:10310000C7010FDC8C01F7018581811521F18091C8
:103110004403909145030097F1F008171907D9F07F
:10312000FC01FF27887F9927892B09F08AC044E09A
:10313000EE0FFF1F4A95E1F7EC53FD4F8581846048
:10314000858311830083CF0190DA10925E0361E0E2
:10315000C701E7DB8C01D70115968C91811509F425
:10316000FAC0C80197578038910508F04AC100316C
:1031700008F0CBC26EE271E080E090E0D8DB811114
:10318000C4C2812C912C540101115EC004E09E0147
:103190002F5F3F4F6901D601E02F1D92EA95E9F7B5
:1031A00024013501FFEF4F1A5F0A6F0A7F0AC5013C
:1031B000B401BDDB8983811509F4A7C2813009F010
:1031C000C7C0A50194012E5F3F4F4F4F5F4F2F8324
:1031D000388749875A87C301B201A9DB182F8A8330
:1031E000811509F492C28FEF810F833008F045C03A
:1031F0006F81788589859A859ADB8B83811511F09B
:10320000C60186DE2401350133E0430E511C611CEA
:10321000711C61C0203E42E5340760F4203852E55D
:10322000350708F06CCFC90180529245809708F0AD
:1032300050CF65CFC90187579C470297F8CF80319F
:10324000F6CFE0E0F0E07ACFBFE28B16B1E09B066C
:10325000A104B10409F459C2C501B40168DBEFEF60
:103260008E1A9E0AAE0ABE0A8111EECF01508CCF93
:103270004F80588469847A842EC08BEF810F83300D
:1032800098F52401350143E0440E511C611C711C6A
:103290006F81788589859A854ADB8B838115D9F082
:1032A000C301B20144DB8C83811571F08B819C8159
:1032B00081305FEF950710F0982F8827163071F056
:1032C000173079F00E94B3252401350134E0430E14
:1032D000511C611C711C530142015DCF0E9471257C
:1032E000F3CF0E949225F0CF143009F0C1CF6F8147
:1032F000788589859A851BDB182F2401350184E0A8
:10330000480E511C611C711CC501B4016D5F7F4FDB
:103310008F4F9F4F0CDB111509F4F7C1811509F48C
:10332000F4C18150990B4FEF489F9001499F300D98
:103330001124A12FA150BB0B2A0F3B1F2150310993
:1033400050F2EFE9FFE03197F1F700C00000F6CF4F
:10335000C601DEDDC0CF680127E5D21AC11431E015
:10336000D30608F497C08091C00380FF45C10E9436
:10337000FD095C01F7018581811509F44FC1809138
:103380001A0182FF05C040E0B50180E090E0C5D899
:103390000431FCE71F0709F43DC105312CE7120792
:1033A00009F4D7C003313CE7130709F418C1C80179
:1033B00090528115904308F0D6C010924B031092A2
:1033C0004A03F7019581911509F4B8C2109253038D
:1033D000980130572332310508F0B0C284E090E004
:1033E0000E949D2F9093CE038093CD03F801E1506E
:1033F000F047E232F10508F0EBC1EB5FFF4C0C94B3
:103400001B2FC80197558115914008F0ACCF58018A
:1034100058EFA522BB24A114B10409F076C1F8012C
:10342000FF2794E0EE0FFF1F9A95E1F7CF018C5331
:103430009D4F6C01D70115968C91E753FD4F9081FC
:1034400080FB90F99083811509F467C00E94FD0903
:103450009093470380934603F60182818F5F8283B6
:1034600080915E0390915B03892B83838091570346
:1034700084834681578166857785C6010E94360917
:10348000D60115968C9181FF5801B0924503A09208
:10349000440369CF6AEB72E08C2D46DC892B09F07E
:1034A000B6CFC60124E0880F991F2A95E1F7FC01E9
:1034B000EC53FD4F2281213029F52091BA02309141
:1034C000BB02232B09F4A3CF2091BC023091BD0293
:1034D000232B09F49CCF2091BE023091BF02409172
:1034E000C0025091C102242B352B232B09F08FCF22
:1034F000FC01E753FD4F20812E7F20838C539D4F8D
:10350000B4D885CF223009F082CF2091BE0230910D
:10351000BF02232B09F47BCFEBCFF6014485558501
:1035200066857785C6010E943609D60115968C916D
:1035300081FF19CFC6017DD8809144039091450346
:103540000817190709F00FCF109245031092440392
:103550000ACF90911A01892F8E7F90FF816080930E
:103560001A010E94701280911A0180FF45C0083232
:10357000110508F069C00E31110508F076C0C801C8
:1035800004974A9788F58091C00384FD2DC0D70128
:1035900015968C91811509F4EAC08091570390919A
:1035A0005B03892B8D7F811509F464C010924B0356
:1035B00010924A038091C00381FD5CC060E0C801A5
:1035C0000E94700860E0C8010E94C90E80915703F4
:1035D0008D7F0E94810A82E00E947B0596C08091C7
:1035E0001A01816080931A01F7018581811521F00C
:1035F00010924B0310924A03D70115968C91F80153
:10360000E851FC47E730F10508F0DBCEE95DFF4CFF
:103610000C941B2F80911A018E7FA1CF80911A01EB
:103620008F7E013E110531F0053E110531F4809188
:103630001A018F7D80931A0196CFC801905281158F
:10364000904308F090CFBDCE0933110558F40D32E8
:10365000110518F40B32110539F68091C00382FD73
:10366000C3CF95CF04361105F7CF8091C00383FDFA
:10367000BBCF8DCF87E0F701ACE4B3E001900D92B2
:103680008A95E1F710924F0310924E0380914A03FE
:1036900090914B030817190709F04CC02091C00303
:1036A00025FF48C030911A0131FF02C026FF42C0F9
:1036B00020914803309149036501C21AD30A49DBBE
:1036C000C816D906B8F580915B0381FF08C08091C8
:1036D0001A01806180931A0182E00E949C0580910A
:1036E0005B0385FF08C080911A01806280931A01F4
:1036F00080E20E949C0560911A016695617080913C
:103700004A0390914B030E94C90E80915F0387701A
:10371000811561F0D70115968C91811539F0809152
:10372000CE0382FF03C082E00E947B052A96E0E17F
:103730000C94462F80915703D0905B03D82AD1FA7E
:10374000DD24D0F88D7F0E94810A10934B030093F3
:103750004A03B0924903A0924803DD0C6894D2F862
:1037600090911A01997FD92AD0921A0134CF40E062
:10377000B501C8010E948D12C8CF06E221EE41EECC
:103780006AE17CE703DBC1CF07E225EE45EE6BE1A2
:103790007CE7F8CF06E221EE40EE68E17CE7F2CF6D
:1037A00007E225EE44EE69E17CE7ECCF06E221EE8C
:1037B00042EE6CE17CE7E6CF07E225EE46EE6DE1F6
:1037C0007CE7E0CF08E221E045EE6EE17CE7DACF6E
:1037D0008091CD0381608093CD038DEC93E00E94B6
:1037E0009C0D0E94380F91CF8091CE03886080930A
:1037F000CE03F3CF8091CD038260EDCF8091CD03D6
:103800008460E9CF8091CD038860E5CF8091CE03BD
:103810008160EDCF8091CE038260E9CF8091CD03AE
:103820008061D9CF8091CD038062D5CF8091CD03C7
:103830008064D1CF0E94380F8091CD038068CBCFB8
:103840008091CD038C60C7CF8091CE038360CFCFB2
:103850008091CD038E7FBFCF8091CE03877FC7CF6E
:103860008091CD038D7FB7CF8091CD038B7FB3CF78
:103870008091CD03877FAFCF8091CE038E7FB7CF6E
:103880008091CE038D7FB3CF8091CD038F7EA3CF68
:103890008091CD038F7D9FCF8091CD038F7B9BCF78
:1038A0000E94380F8091CD038F7795CF8091CD0303
:1038B000837F91CF8091CE038C7F99CF8091CD0370
:1038C000992782FF939590FB82F990FB83F983CF30
:1038D0008091CE03982F909590FB80F990FB81F911
:1038E00086CF9091CD03892F8F7B96FF806473CF15
:1038F0000E94380F9091CD03892F97FB87F980584C
:103900006ACF61E08EE090E00E94B12F66CF60E068
:10391000F9CF9091CD03892F8F7E94FF80615BCF8B
:103920009091CD03892F8E7F90FF816054CF90912D
:10393000CE03892F877F93FF886059CF0631FCE73C
:103940001F07D1F580915B033091BF0330FF04C0A6
:10395000282F2474211124C0282F2A7A31FF04C073
:10396000482F4171411120E032FF04C0482F4878B0
:10397000411120E033FF03C08272811120E09115D4
:1039800089F081E0211101C080E08093540385E338
:10399000211101C089E20E949A090E94DC0DB5CE76
:1039A00020E0DCCF80915403811521F085E30E9453
:1039B000CE09F3CF89E2FBCF07372CE71207F9F0E6
:1039C00008373CE7130731F19801205E3245203279
:1039D000310528F591113BC00F7181E090E0AC01F9
:1039E00002C0440F551F0A95E2F78A01642F83E055
:1039F00090E00E94B12F802F0E94590486CE81E072
:103A0000911551F00E945F0443E062E081E00E9462
:103A1000E1047BCE82E0F4CF0E946904F5CF9115DA
:103A2000B1F00A355CE7150709F493C008F06AC0E5
:103A300001309CE7190709F48AC00330ACE71A0784
:103A400009F47FC00115BCE71B0709F46DC0F7013D
:103A50008581C080D180811509F47FC0C6010E9494
:103A60003314182F682FC6010E947704B601812FE6
:103A70000E9418140E94A206182FD92E86E0F70182
:103A8000DE01119601900D928A95E1F7D701159606
:103A9000CC9015971696BC90B2948FE0B822809186
:103AA0005F038770811501F1AC2CC114F1F0892FEF
:103AB000807F803461F080E2810F8830A8F0892F08
:103AC000807E803221F4123078F0B11469F0809158
:103AD000CE0382FF09C082E00E947B0580915F03D4
:103AE0008770AA24A3948111A12C8D2D82958F70AB
:103AF000882E912C8C3008F04FC0F401E25DFF4C11
:103B00000C941B2F0B35ECE71E0729F18091CE0397
:103B1000002482FF0394802D0C35FCE71F0709F079
:103B200096CF0E94A30D93CF0E94380F2FEF34E35E
:103B30004CE0215030404040E1F700C000000E94BE
:103B4000110D6FEF7FEF80E090E00E94CB2F0E947D
:103B5000640F81E0E6CF80E0E4CFC6010E94AD04AF
:103B6000182F84CF0D2D0F70B0E1DB1610F00295E9
:103B7000007FC11409F44AC0011559F080E2810F99
:103B8000883010F011113CC0802F0E9496050E94D1
:103B9000DC0D812F0E944F0EE8E08E1A9108F4E0B0
:103BA0008F16910418F40E943B09A12C812F9D2DA2
:103BB0000E943504811541F0C11409F413C2B114F7
:103BC00009F407C21092D103A114A9F080915F03F8
:103BD00080FD11C0D70115961C9286958695869515
:103BE0000E945F04C7013DDA80915F038695869548
:103BF00086950E94690460E0C7010E94911496CDE9
:103C000080915E03802B80935E03C1CF812F0E9441
:103C1000D70E011509F4C0CF80E2810F883010F073
:103C2000111104C0802F0E949C0506C00095809150
:103C30005E03802380935E030E94DC0DADCF0D2DCB
:103C40000F708D2D807F803211F00295007F11154D
:103C500049F0113009F473C0C11409F47FC0B114E4
:103C6000D9F097CF8091CE0382FD12C0C11449F0E4
:103C7000011529F0802F0E9496050E94DC0D80E03E
:103C800089CF80E00E94D70E011509F485CFCACFF5
:103C9000C11491F1B11004C0802F0E94300E7CCF6E
:103CA00021E0B21211C070905703802F87210817AE
:103CB00009F472CF0E94FD09909356038093550337
:103CC000702A7092570368CF8091C103823008F444
:103CD00063CFB81261CF802F0E94300E802F0E94D8
:103CE0006C0A80915803902F9823091709F454CF38
:103CF000802B8093580350CFB11012C0802F0E94A8
:103D00003F0E802F0E946C0A80915803902F9823B9
:103D1000911509F441CF00950823009358033CCF37
:103D20008091C103823008F437CF31E0B31234CF31
:103D300080915B038023811509F42ECFDFCF809122
:103D4000C703C11421F08B1508F426CFA5CFB816F0
:103D500008F022CF802F0E943F0E1ECFB114D1F366
:103D60008091C5039091C603193321F08091C3035C
:103D70009091C4030E94030D812F0E94D70E0CCF97
:103D80008D2D869586958370811569F0813009F0B7
:103D900003CF812F9D2D9370C11002C080E090E071
:103DA0000E947209F9CE812F9D2D9370C11002C01F
:103DB00080E090E00E944A09EFCE6C2D812F0E9496
:103DC000BD0AEACE8D2D8370811133C0C110E4CEBF
:103DD000412F429546954770440F440F812F8F70B5
:103DE000042E01C0880F0A94EAF7212F207114FFD6
:103DF00007C02FE030E001C0220F4A95EAF7209576
:103E00003D2D369536953370323071F0333051F0A8
:103E100040915903313029F0822B84230E945904A8
:103E2000BBCE842B822BFACF822B9091590389270A
:103E3000F5CFC11459F1D0FEAFCE412F4295469532
:103E40004770440F440F812F8F70042E01C0880FDC
:103E50000A94EAF7212F207114FF07C02FE030E009
:103E600001C0220F4A95EAF720953D2D36953695EB
:103E70003370323089F0333069F040915A03313079
:103E800041F0822B84230E945C0486CE8230A8F607
:103E900083CE842B822BF7CF822B90915A038927D4
:103EA000F2CF0D2D0F70C11429F0802F0E945F04F6
:103EB000812FF3CE812F0E943F0E802F0E94690434
:103EC0006BCE123F71F160F4103FB9F0113F81F0F9
:103ED000C11409F479C0B1105CCE8D2D8F7125C04D
:103EE000133F31F1143FA1F78091CE0382FD2CC026
:103EF0008D2D8F71C11411F318C08091C703C114A7
:103F000061F0B81608F048CE2D2D2F7181E090E0B9
:103F100001C0880F2A95EAF7C0CF8B1508F43CCE74
:103F2000F3CF8D2D8F71C110C9CF0E945F0434CEA5
:103F300080E0C11409F4A7CF81E09D2D9F7101C0DD
:103F4000880F9A95EAF79FCF8091C103823048F19C
:103F5000C114C9F090915F039770943059F4109296
:103F60005F0310926103109260038D2D8F710E9488
:103F7000690419CE63E0B81608F015CE8D2D8F7147
:103F80000E94580A10CEB81640F010925F031092AB
:103F900061031092600364E0F1CF81E00E947B0531
:103FA00002CEC11431F063E08D2D8F710E94580A4A
:103FB000F3CD81E00E947B0542E0B41608F4ECCD1D
:103FC00082E00E947B05E8CDB110CACE8D2D8F71A5
:103FD00075CF80915D0380935C0380915B03809338
:103FE0005D03F2CD40E060E089819A810E94751402
:103FF0009C0100915B03B11429F01092D10300934E
:104000005D03E2CD8091CF039091D003281739074B
:10401000B1F78091C20382FFF0CF8091D103811567
:1040200061F380915C030E94300E812F0E942D0F5E
:1040300080915C030E943F0EE0CFA0E0B0E0E3E29D
:10404000F0E20C94332F8091A403803108F049C032
:104050008091A303811509F444C0C091650387E0F2
:10406000D82E809164038C17E1F1EC2EF12CDC9EAC
:10407000E0011124FE01EA59FC4F84818115B1F160
:10408000918180919F03981331C0908180919E030C
:1040900098132CC08581811129C0028113818091E0
:1040A000A0039091A103081B190B60E08EE993E037
:1040B0000E9491140E94A91608171907B8F480915C
:1040C000A4038F7080618093A403C459DC4F88815E
:1040D0008F70806188838EE993E00E9431180E947E
:1040E0007105CDB7DEB7E7E00C944F2FE7012196BD
:1040F000C770B7CFCF92DF92FF920F931F93CF93EA
:10410000DF93182F092F87E0F82EC0916503809167
:104110006403C81799F1FC9EE0011124CE018A596D
:104120009C4F6C01FC018581811589F0C6010E94BC
:104130006A14811561F0FE01E459FC4F20812F7053
:1041400020612083F601808191810E94790FC60150
:104150000E9431182091650330E02F5F3F4F277098
:10416000332720936503CA59DC4F89818013CDCF53
:1041700088818113CACF8D81811539F2DF91CF916A
:104180001F910F91FF90DF90CF900895EF92FF92D3
:104190001F93CF93DF93EC0120911B01211541F078
:1041A00010E0812FDF91CF911F91FF90EF90089544
:1041B000EA80FB80E61AF70A24EFE21621E0F20615
:1041C00078F760E0CE010E9491149C0130522115D5
:1041D000304330F70E943C05811511F38091B802FD
:1041E0009091B9020E943C05182F8115C9F2809167
:1041F000CB039091CC03853F21E0920710F084EF30
:1042000091E0E816F90660F68E818F7080618E83EA
:10421000888199810E94790F0E940005CE010E9439
:104220003118BFCFADE0B0E0E8E1F1E20C94292F06
:104230008C0186E0F801DE01189601900D928A95B6
:10424000E1F7D8014C9011963C9011971296ED90A1
:10425000FC90139714965C90149715966C906110CF
:104260000CC050919302252F30E0E0E08E2F0E2EEF
:10427000000C990B821793073CF15EE9A52E53E0E1
:10428000B52E8091A203811151C05114D1F0611457
:1042900009F413C3C8010E946A14811509F40DC3FF
:1042A0006091620370916303C80170DF811109C0DE
:1042B00087E0F801AEE9B3E001900D928A95E1F74D
:1042C000BCDEFF24F3948CC0880F991F8D579D4F3F
:1042D000DC0111964C911197431103C08C91481643
:1042E00011F0EF5FC3CFEF3F41F2D80116968C91EA
:1042F00016978F70806116968C93E517A0F4AFEF38
:10430000A50FA0939302EA1770F4F0E0EE0FFF1FE1
:10431000ED57FD4FB0E0AA0FBB1FAD57BD4F8D91BC
:104320009C91918380830E940005A7CF60E08EE975
:1043300093E00E9491146C017090A3038091A003FC
:104340009091A1034701881A990A60E08EE993E0F1
:10435000711409F456C20E9491140E94A91688167D
:10436000990608F00CC2511409F4ABCF80919F0359
:10437000F8019181B090A403F0E1BF1608F0C8C124
:10438000981350C090919E03D8018C9198134AC005
:10439000611048C08B2D8F7080618093A4038EE9DB
:1043A00093E00E9431188091A403F8018683F09075
:1043B000A003E090A10347E0D42E00916503809113
:1043C0006403081751F0D09E800111240A591C4F34
:1043D000D80115968C91811108C00E947105F12CAD
:1043E0008F2D2D96E1E10C94452FF801B280C3800A
:1043F000C8010E946A1481110EC0C8010E943118C0
:104400008091650390E001968770992780936503FA
:10441000FB2CEC2CD2CF6F2D7E2DC801B7DE811185
:10442000EFCFDBCFF0E2DF1AC11420E3D20608F0B1
:1044300084C0611005C140E0632D842D0E94E40C0E
:1044400081114FC040E0632D842D0E94E40CF82EB2
:10445000811509F429C18091C20380FFC0CF8EE984
:1044600093E00E94311860E08EE993E00E9491147D
:104470008C01F09065037F2C98E0E92E2EE9822EC6
:1044800023E0922E37E0432E809164037816A1F04A
:10449000A72CB12C479CC0011124FC01EA59FC4F08
:1044A0006F0160E0CF010E949114582E692ED60151
:1044B00015968C91811197C0B8E0EB1618F417E0AF
:1044C000EF10ACC08885998515DE0E9400050E941A
:1044D000710587E0EEE9F3E0DF011D928A95E9F7C7
:1044E0007ECF60E0C8010E9491148091C20383FFD7
:1044F000A9CFB8018EE993E00E940D058111A2CFEA
:104500008091A4038F7080618093A40380919E03A7
:1045100090919F030E94790F8EE993E00E943118D9
:10452000EEE9F3E087E0DF011D928A95E9F78885DF
:104530009985E0DD0E94000550CF611409F482CF17
:104540008091A40381608093A4038091C20381FFC2
:1045500046CF8EE993E00E94311800916503809167
:104560006403081709F4CCC0E02EF12CB7E00B9FD0
:10457000C0011124FC01EA59FC4F6F01CF010E94D8
:104580006A14811509F4BCC087E0F601AEE9B3E016
:1045900001900D928A95E1F7C701019687709927DE
:1045A000082F809365030E94710587E0F82E8091A3
:1045B0006403801709F411CFF09E800111240A5979
:1045C0001C4FC8010E946A14811107CFC8010E94C4
:1045D00031188091650390E0019687709927082F24
:1045E00080936503E4CF10520115E0E31E0708F045
:1045F00063CF8091C20383FD0AC0E72CC5010196F9
:10460000F82FF7707F2E052D162D46013DCFB601F0
:10461000C4010E940D05811589F3EFCF1F9DC001D4
:1046200011248A599C4F0E9431182091650330E073
:104630002F5F3F4F27703327F22E2093650340CF23
:104640008091A40381608093A40360E0C8010E946C
:1046500091148091C20383FF78CFB8018EE993E073
:104660000E940D05811171CFF090A403E894F0F839
:10467000F092A403C8010E946A148111B0CE8F2D5C
:104680008F7080618093A40380919E0390919F031B
:104690000E94790F0E9400058EE993E00E94311874
:1046A000EEE9F3E087E018CF888599850E945D14D4
:1046B000292F22952F70903450F49F70223080F073
:1046C000911599F0F8019681903178F489CE2A5F9E
:1046D0002F70223078F0C8010E943118F72C80CE5C
:1046E000911519F0811509F47BCE805E883008F4AD
:1046F00077CEF1CF803F08F473CE815F8330F7CF60
:1047000087E0EEE9F3E0DF011D928A95E9F74DCFEE
:10471000981315C090919E03F801808198130FC0E3
:1047200061100DC0B682C8010E94311887E0F801FF
:10473000AEE9B3E001900D928A95E1F7C2CDC801D0
:104740000E946A14811509F4B8C0611409F4B5C057
:104750008091A403803208F4ABCD80919E039091A8
:104760009F039A838983FC82EB828091A2038D83CD
:104770001E82BF82CE0101960E94311899CDD09041
:10478000A403F0E1DF1638F48EE993E00E943118BB
:1047900087E0D501A2CE511409F493CD90919F03E7
:1047A000F8018181981311C090919E038081981324
:1047B0000CC061100AC0D682C8010E94311887E07F
:1047C000D5011D928A95E9F77CCDC8010E946A1433
:1047D000811509F472C0611409F46FC08091A403BB
:1047E000803208F465CD80919E0390919F039A8357
:1047F0008983FC82EB828091A2038D831E82DF82FB
:10480000B9CF0E9491140E94A9168816990608F043
:1048100058C0511409F455CD611409F44EC090915B
:104820009F03F8018181981330C090919E0380818D
:1048300098132BC08091A0039091A103E81AF90A64
:1048400060E08EE993E00E9491148091C9039091F9
:10485000CA03E816F90608F069CF8091A40380FD29
:1048600065CF803108F462CFD80116968C931697E5
:10487000982F907F903F09F456CF982F907F905FAC
:104880008F70892B16968C934ECFC8010E946A14A4
:10489000811571F06091620370916303C80176DC49
:1048A000811509F405CD87E0EEE9F3E0DF0189CF5A
:1048B0008091A40381608093A403C8010E943118F1
:1048C00000CD87E0F50111928A95E9F788CDABE13B
:1048D000B0E0EDE6F4E20C94342F4E8B5F8B688FE2
:1048E000798F082F8A8F192F9B8FF82EE92E81152B
:1048F00009F4A1C040E0692F8E899F890E94751438
:104900009C01111549F01092D1039093D00380932C
:10491000CF0310925E030AC08091CF039091D00321
:104920008217930719F481E08093D1031D8A86E0F2
:10493000FE017696DE011F9601900D928A95E1F7B1
:104940008091CE0382FF21C08091A7039091A8039C
:10495000892BD9F00E94FD092091600330916103F9
:10496000821B930B2091A7033091A8038217930712
:1049700038F080915F0382FD03C082E00E947B05D6
:104980000E94090A81110E94A405F11461F00B8BA9
:104990001C8B61E0CE010F960E94911461E0CE0164
:1049A0000F960E9491140B8B1C8B87E0FE013F96A3
:1049B000DE01189601900D928A95E1F7CE010896D6
:1049C00031DC811110C0209164033091650387E0D0
:1049D000FE013896DE01119601900D928A95E1F75D
:1049E0008C8581112CC017E0809165039091640340
:1049F000891741F0189FC00111248A599C4F12DC7D
:104A0000811144C08C85811112C080911B018111DC
:104A10000EC08A859B852091620330916303821BBF
:104A2000930B8F3F9F4318F081E080931B016B969F
:104A3000E6E00C94502F911509F478CF6ACF822FBD
:104A400090E00196877099273817190671F40E9433
:104A5000380F109264031092650387E0EEE9F3E0EB
:104A6000DF011D928A95E9F7BECF97E0929FD001B2
:104A70001124AA59BC4FFE01319601900D929A95CE
:104A8000E1F7809364030E947105ADCF80916503C7
:104A900090E001968770992780936503A5CFA6E0E3
:104AA000B0E0E5E5F5E20C94362F0E94FD098C019B
:104AB00080915702909158028017910771F01982E6
:104AC0001A820E94FD09BC0149815A8180E090E070
:104AD000FEDE10935802009357022696E4E00C94F1
:104AE000522FA6E0B0E0E7E7F5E20C94382F909360
:104AF000540280935302811520E2920730F40E9401
:104B0000B40E2696E2E00C94542F80EF89838A83BA
:104B10000E94FD098160BC0149815A8181E091E0D8
:104B2000D6DEEFCFA6E0B0E0E8E9F5E20C94382F4E
:104B30009093540280935302811520E2920730F43F
:104B40000E94020F2696E2E00C94542F80EF898396
:104B50008A830E94FD098160BC0149815A8181E0FC
:104B600090E0B5DEEFCFCF93DF93D82FC92FB9DF19
:104B70008091C3039091C4030E94030D8D2F9C2F3D
:104B8000D1DFDF91CF9108950F931F93CF93DF93E0
:104B90008C01862F6AEB72E00E949416892B91F4A7
:104BA000C091BA02D091BB02209761F0F8018281D6
:104BB000833039F4CE01D7DFCE01D5DFCE01D3DF8C
:104BC00001C0E0F7DF91CF911F910F9108950F93EE
:104BD0001F93CF93DF938C01EB016AEB72E08C2F74
:104BE0000E949416892B09F057C0FE01FF27D801B7
:104BF00012968C911297E25EFD4F8130A9F41596C2
:104C00008C9182FD4EC080FF4CC082E080838091F9
:104C1000BC029091BD020097B9F48091BA029091C4
:104C2000BB020097C9F110C08230A1F515968C9196
:104C300082FD26C080FD0AC083E080838091BE0291
:104C40009091BF020097F1F04CDF26C084E0808392
:104C50008091C0029091C1020097B1F78091BA0291
:104C60009091BB02009701F17EDF8091BC02909190
:104C7000BD02009749F78091BA029091BB02E4CF40
:104C800085E080838091BA029091BB02009721F069
:104C90006ADFF1CF86E08083DF91CF911F910F9182
:104CA000089581E08083B9CF8091BC029091BD02CC
:104CB000B8CF0F931F93CF93DF938C01EB016AEB77
:104CC00072E08C2F0E949416892BA1F48091C3036B
:104CD0009091C4030E94030DDD27C25EDD4F8881E1
:104CE000F801128218828330E9F048F4813059F0DB
:104CF000823081F0DF91CF911F910F910895843020
:104D0000B1F08530B9F78091BA029091BB0200975B
:104D100089F306C08091BC029091BD02009799F37F
:104D200001DFE8CF8091BE029091BF02F7CF809162
:104D3000C0029091C102009799F72091BA02309178
:104D4000BB028091BC029091BD0221153105F9F2A0
:104D5000009731F7C901E4CFCDB7DEB7AC970FB6F6
:104D6000F894DEBF0FBECDBF85B7806885BF85B71D
:104D7000806885BF84B7877F84BF0FB6F894A895F5
:104D800080916000886180936000109260000FBE87
:104D900080E890E00FB6F8948093610090936100F2
:104DA0000FBE81E0809319018EE997E09093B501E1
:104DB0008093B4010E94B9070E9477130E942D0CC2
:104DC0000E948A0C8091E20084608093E2007894D3
:104DD00080915202811599F08091E9001091EC00C8
:104DE0008F70179511271795182B1092E900809155
:104DF000E80083FD0E94AD0F1F701093E90082E070
:104E000084BD93E095BD9AEF97BD80936E000E949C
:104E1000A814811102C00E94631704E311E0D801B5
:104E20008D918D018F3F11F00E94A007B1E00933F1
:104E30001B07A9F709E311E0F80181918F018F3F6A
:104E400011F00E94A007F1E007341F07A9F78AE0DC
:104E5000E6E4F2E0DF01282F1D922A95E9F7E6E269
:104E6000F2E0DF011D928A95E9F780E090E00E9470
:104E70009D2F833E9E4F21F40E94A81481112AC0C9
:104E800063EE7EEF80E090E00E94CB2F60E082E056
:104E900090E00E94B12F81E08093590361E083E0AC
:104EA00090E00E94B12F198284E18A83CE0101969D
:104EB0000E949C0D0E94631740E050E0BA018FE011
:104EC00090E00E94C32F40E050E0BA0183E190E0FF
:104ED0000E94C32F82E090E00E94952F80933202BF
:104EE00084E090E00E949D2F9093CE038093CD03A9
:104EF0000E94E415EFEBFDE53197F1F700C00000EB
:104F00000E94E4158091460280FF08C06FEF7FEF9A
:104F100080E090E00E94CB2F0E94110D83E090E092
:104F20000E94952F0E94590484E091E090937A02A8
:104F30008093790280915202853049F48091520227
:104F4000853009F45CC00E94380F0E943B090E9422
:104F5000E415F3E3AF2EF2E0BF2E06E412E0D80131
:104F6000F501219131918D919D914DE352E04E17C4
:104F70005F0709F47AC02817390799F3E6E48E2E03
:104F8000E2E09E2E512CD401ED90FD904D01F501F3
:104F9000619071905F016E147F0451F16E247F2443
:104FA000412CCC24C394D12CC3018C219D21892B6D
:104FB000B1F049825A820E94FD099C838B83F1E003
:104FC000FD8391E097012C213D21232B09F490E0F2
:104FD0009E8349815A816B817C818D8178DC4394E9
:104FE000CC0CDD1C2EE04212DFCFF501F292E292F2
:104FF000539435E05312C7CF0E94780B3BC0809189
:105000005202843021F11092300228E130E040E475
:105010000FB6F894A895209360000FBE40936000EF
:1050200083B7817F846083BF83B7816083BF7894B7
:10503000889583B78E7F83BF0FB6F894A89580912B
:105040006000886180936000109260000FBE0E9433
:10505000E415E6E4F2E081919191892B09F0FBC41B
:1050600052E0E035F507B9F769CF2817390709F09D
:1050700085CF15DDC0904403D0904503C114D10401
:1050800039F1A0904603B09047030E94FD097C01CE
:10509000EA18FB08C6010E94A9168E159F05C0F4E8
:1050A0002091440330914503C9019927287F332774
:1050B000232B09F090C054E0880F991F5A95E1F70F
:1050C0008C539D4FDC0115962C9122FF0E943513C5
:1050D0008091C00380FF1CC080911A0182FF18C01C
:1050E0000E94FD09BC0180914803909149039B01F6
:1050F000281B390B80911001909111012817390755
:1051000038F041E080914A0390914B030E948D1248
:1051100086E0E2EBF2E0DE01119601900D928A95B5
:10512000E1F79090B302B090B402E090B502A09085
:10513000B602F090B7021092B4021092B50210922B
:10514000B6021092B7028E2D8B29811509F44FC03B
:10515000C0903F02D09040020E94FD099C012C1992
:105160003D099091B0029115C9F180911501821706
:105170001306E8F59F3F19F09F5F9093B002B114BA
:1051800059F00E94A40891E01B140CF09FEF899F36
:10519000802D11248093B402E11459F00E94A408D8
:1051A00091E01E140CF09FEF899F802D11248093B5
:1051B000B5028091B4028115D1F0D090B502D1141E
:1051C000B1F00E9496088093B4028D2D0E9496083B
:1051D0008093B5020CC080E090E074CF4091140140
:1051E000BAE04B9FA00111244217530728F28F2DDC
:1051F0008A29811509F44CC0C0903D02D0903E022E
:105200000E94FD099C012C193D099091AF02911556
:10521000B1F18091130182171306D0F59F3F19F069
:105220009F5F9093AF02A11459F00E94FD0891E096
:105230001A140CF09FEF899F802D11248093B602E1
:10524000F11459F00E94FD0891E01F140CF09FEF3B
:10525000899F802D11248093B7028091B602811519
:10526000B9F0D090B702D11499F00E9496088093BB
:10527000B6028D2D0E9496088093B70209C0409116
:105280001201EAE04E9FA00111244217530740F299
:105290008091B302891119C08091B402811511F077
:1052A0008B1113C02091B502211511F02E110DC0E4
:1052B0009091B702911511F09F1107C03091B6027D
:1052C000311103C0822B892B81110E94940A86E040
:1052D000FE013196A2EBB2E001900D928A95E1F7C2
:1052E0000E943B0990914102891721F0809341026D
:1052F0000E94780B80915202843009F01BCE83E02B
:105300008093E9008091E80082FF14CE8091E8004C
:1053100090E085FF05C00E94FC0B811519F191E01A
:105320008091E8008B778093E800911509F402CE14
:10533000E0905502F0905602E981E114F10489F100
:10534000EE3F09F04FC08A81833020F085508330D2
:1053500008F048C0EA81EE3008F044C0F0E0E65CB6
:10536000FF4C69C540E2C42ED12C9E012F5F3F4FF8
:1053700079018091E80085FD0AC08091E8008B7773
:105380008093E8000E94FC0B811599F3C8CF8091AF
:10539000F100D7018D937D01B1E0CB1AD10849F717
:1053A000BECFE43148F4E11549F0E150E33130F487
:1053B000F0E0E85BFF4C3FC5EE3F61F28FEF77C353
:1053C0001A8289E08B830EC08A81823081F083301B
:1053D000B1F0813099F70E94780B33D56B837C83D1
:1053E0008D839E83CE0101960E944C0CA3CD88E252
:1053F00090E09BD51B821C821D828E83F3CF80910F
:10540000500290915102892B69F3FE013196D80127
:105410008C9111969C910E5F1F4F928383833296DD
:10542000B2E000351B0799F7DDCF8A81823031F673
:105430006B817C818D819E8104D588E290E091D53D
:10544000D1CF4C816B818A810E94E91398278927EB
:1054500098279E838D83C6CF2D813E8132272327B7
:1054600032274C816B818A810E94B50DBBCF0E948F
:10547000C114B8CF80E18A83B5CF81E08A838FE2FF
:10548000A1CF8C818D3108F0ADCF8A809B8098248C
:1054900089249824A12CB12C8E010F5F1F4F780115
:1054A000E80EF11CE016F10609F49CCF80E0EFE273
:1054B0008E16E1E09E06A104B10420F4C4018F52CF
:1054C0009D4F33D5D80114968C930F5F1F4FBFEFBC
:1054D0008B1A9B0AAB0ABB0AE5CF809150029091D0
:1054E0005102892B09F47ECF8C818D3108F07ACF5F
:1054F000882E912CA12CB12CCA80DB80DC24CD24F9
:10550000DC24E12CF12C8E010F5F1F4F412C512C1C
:105510003201481459046A047B0408F063CFEFE2B7
:10552000CE16E1E0DE06E104F10438F4D801149669
:105530006C91C6018F529D4F14D5BFEF4B1A5B0A79
:105540006B0A7B0AEFEFCE1ADE0AEE0AFE0A0F5F45
:105550001F4FDFCF0E94281745CF84E08CCF8C816E
:105560008D3108F03FCF882E912CA12CB12CCA8010
:10557000DB80DC24CD24DC24E12CF12C412C512CCB
:1055800032018E010B5F1F4F481459046A047B04DB
:1055900008F028CF80E0F0E3CF16F2E0DF06E10468
:1055A000F10418F4C6018996C0D4D8018D938D01F9
:1055B000BFEF4B1A5B0A6B0A7B0AEFEFCE1ADE0ACB
:1055C000EE0AFE0AE1CF2C81022F10E02D3108F007
:1055D00009CF8A819B819827892798272C01612CE4
:1055E000712C8033F2E09F0708F0FCCE822E912CC4
:1055F000A12CB12C40E352E060E070E04419550961
:1056000066097709421751056105710508F4EACE6C
:105610002091500230915102232B09F03EC01C0111
:1056200029E2220E311C80FBEE24FF24E0F880FFEB
:105630000BC088967AD49D81892798278927811560
:105640009C4711F48FEF8D83D501C401840D951D06
:10565000A61DB71D80FF19C0680141E0C41AD1081A
:10566000CE0105968C0D9D1D9CA78BA7C101800FB7
:10567000911F5BD4ABA5BCA59C9181159C4721F4DF
:105680008FEFEBA5FCA580838601FE013196EE0D20
:10569000FF1D2FEFE016F10638F08E010F5F1F4F50
:1056A000C12CD12C760125C09481858181159C4720
:1056B00011F42483258342E0E40EF11C3296EACFF4
:1056C00050E3451652E055066104710430F4D801E8
:1056D00014966C91C201899644D4BFEFCB1ADB0AB1
:1056E000EB0AFB0AEFEF4E1A5E0A6E0A7E0A0F5FA4
:1056F0001F4FC814D904EA04FB0410F373CE809141
:10570000500290915102892B09F46CCECE01019682
:105710000E944C0CFFEF21EE34E0F150204030406D
:10572000E1F700C00000F8CB88E0ECE1F1E0DE0139
:10573000919601900D928A95E1F7FE0132968FE1E4
:10574000DF011D928A95E9F786E0898388E07F96DC
:10575000DE01159601900D928A95E1F743CE8CE417
:10576000898381E08A831B821C823CCE8B819C8151
:10577000092E000CAA0BBB0B35E0880F991FAA1F3E
:10578000BB1F3A95D1F7AC01BD01405E5F4F6F4F33
:105790007F4F481759076A077B0708F423CE8C34DC
:1057A000E1E09E07A105B10508F01CCE4D34F1E003
:1057B0005F076105710520F04CE451E060E070E0A6
:1057C000481B590BBC01635F794FCE01019677D31B
:1057D00009CE4AE150E06FEF70E0CE0107968ED31C
:1057E000809150028983EA821B821C8282E08D8331
:1057F0008DE003CE81E090E09093560280935502B5
:1058000082E390E090934502809344020E94FD0958
:105810009093430280934202E5CDE114F10481F1BB
:10582000D0904602C0904B02009142021091430278
:105830000E94FD09801B910B8536910540F1C5FE44
:1058400026C0D0FE24C00E94FD099093430280939D
:105850004202809144029091450201979093450243
:1058600080934402892B61F41092560210925502E3
:1058700081E090E09093510280935002E12CF12C52
:10588000809150028983EA82809144029BCD82E319
:1058900090E09093450280934402F2CF109251021F
:1058A000109250029FCD0B811C8140E250E06FEFBF
:1058B00070E0CE01019622D325ED34E042E050E0C5
:1058C00080E090E0F901659175910617170740F4A3
:1058D000DE0111968A0F9B1FFC0171836083CA0150
:1058E000F6E021303F0709F47DCDAC014E5F5F4FFC
:1058F000245F3F4F4132510528F374CD2B813C8109
:1059000085ED94E0FC01459155912417350709F484
:10591000BFC00C9646E08D309407A1F74FCD8B8128
:105920009C8105ED14E0F8012591359182179307CC
:1059300009F4BFC0045F1F4FF6E00D301F0799F751
:10594000EE24EA94FE2CD0C00E949D134BCD8B8197
:10595000813069F0823011F1811144CDFE0132961F
:105960008FE1DF011D928A95E9F788E0A0C08C8164
:105970009AE0F92E8E010F5D1F4FF8012F2D119225
:105980002A95E9F7B8010E9494168983F801DE018F
:10599000129601900D92FA94E1F724CD6C818AE081
:1059A000FE013596DE01919601900D928A95E1F700
:1059B00089A19AA181153CE7930741F420915002F7
:1059C00030915102232B11F480E090E09AA389A337
:1059D0008BA19CA181154CE7940741F420915002C2
:1059E00030915102232B11F480E090E09CA38BA313
:1059F0008DA19EA181155CE7950741F4209150028D
:105A000030915102232B11F480E090E09EA38DA3EE
:105A10008FA198A58115ACE79A0741F42091500217
:105A200030915102232B11F480E090E098A78FA3CE
:105A30008FEF683060F4BAE06B9FB00111246F57AC
:105A40007D4F4AE050E0CE018196A9D280E0898363
:105A50000E94B907C7CC80913102811509F46ECA42
:105A600080E189BD92E199BD09B400FEFDCF80912E
:105A7000D8008F7D8093D8008091E0008260809371
:105A8000E0008091E00081FDFCCF0E94380F56CAF3
:105A9000FC013696259135912115310509F48ECCFE
:105AA0004FE150E0BE016E5F7F4FF9010995898398
:105AB00099CCF8013896259135912115310509F4D5
:105AC0003FCF4CE150E0BE016B5F7F4FC801F90151
:105AD00009957C01892B41F4F8013A9685919591BD
:105AE000009711F0FC010995E9827CCC1F921FB64A
:105AF0001F9211248F939F93AF93BF938091300295
:105B0000811113C08091F6019091F701A091F801E5
:105B1000B091F9014196A11DB11D8093F6019093BA
:105B2000F701A093F801B093F901BF91AF919F9154
:105B30008F911F901FBE1F90189578941F921FB6CB
:105B40001F9211248F939F93AF93BF938091F6017F
:105B50009091F701A091F801B091F9010196A11D72
:105B6000B11D8093F6019093F701A093F801B093D3
:105B7000F901BF91AF919F918F911F901FBE1F9010
:105B800018951F920F920FB60F9211242F933F93E7
:105B90004F935F936F937F938F939F93AF93BF9335
:105BA000EF93FF938091E10082FF09C08091E200B2
:105BB00082FF05C08091E1008B7F8093E10080919E
:105BC000DA0080FF24C08091D80080FF20C080913F
:105BD000DA008E7F8093DA008091D90080FFA9C01F
:105BE00080E189BD82E189BD09B400FEFDCF81E07D
:105BF000809352028091E501811109C00E942D0C11
:105C00000E948A0C8091E20084608093E20080917F
:105C1000E10080FF1AC08091E20080FF16C08091F1
:105C2000E2008E7F8093E2008091E20080618093A9
:105C3000E2008091D80080628093D80019BC85E092
:105C40008093520283E0809319018091E10084FFE8
:105C50002FC08091E20084FF2BC080E189BD82E1EA
:105C600089BD09B400FEFDCF8091D8008F7D80935F
:105C7000D8008091E1008F7E8093E1008091E20066
:105C80008F7E8093E2008091E20081608093E20049
:105C90008091E401811509F452C084E0809352029E
:105CA00080915202843009F052C082E08093190141
:105CB0008091E10083FF2CC08091E20083FF28C027
:105CC0008091E100877F8093E10082E0809352021F
:105CD0001092E4018091E1008E7F8093E100809139
:105CE000E2008E7F8093E2008091E20080618093E9
:105CF000E20042E060E080E00E945A0C8091F000F7
:105D000088608093F00081E08093190180931801EE
:105D1000FF91EF91BF91AF919F918F917F916F9183
:105D20005F914F913F912F910F900FBE0F901F9059
:105D3000189519BC109252021092E50168CF80911B
:105D4000E30087FF02C083E0A9CF81E0A7CF81E015
:105D5000ADCF1F920F920FB60F921124EF92FF92C8
:105D60000F931F932F933F934F935F936F937F9363
:105D70008F939F93AF93BF93CF93EF93FF9309EECE
:105D800010E0F8018081C091EC008F70C795CC279E
:105D9000C795C82B108280EFE82EF12CF701808187
:105DA000877F808378940E94AD0FF8011082F701FD
:105DB000808188608083CF70F801C083FF91EF916C
:105DC000CF91BF91AF919F918F917F916F915F9193
:105DD0004F913F912F911F910F91FF90EF900F9056
:105DE0000FBE0F901F901895AA1BBB1B51E107C057
:105DF000AA1FBB1FA617B70710F0A61BB70B881F5B
:105E0000991F5A95A9F780959095BC01CD010895E9
:105E100097FB072E16F4009406D077FD08D0E4DF38
:105E200007FC05D03EF4909581959F4F089570959D
:105E300061957F4F0895EE0FFF1F0590F491E02DBF
:105E4000099469279627692778278727782708954F
:105E50002F923F924F925F926F927F928F929F927A
:105E6000AF92BF92CF92DF92EF92FF920F931F9368
:105E7000CF93DF93CDB7DEB7CA1BDB0B0FB6F89419
:105E8000DEBF0FBECDBF09942A88398848885F8459
:105E90006E847D848C849B84AA84B984C884DF80CA
:105EA000EE80FD800C811B81AA81B981CE0FD11DAE
:105EB0000FB6F894DEBF0FBECDBFED010895FB0114
:105EC000DC0102C005900D9241505040D8F7089572
:105ED000FB01DC0104C08D910190801921F4415037
:105EE0005040C8F7881B990B0895FB01DC0102C0E4
:105EF00001900D9241505040D8F70895DC0101C047
:105F00006D9341505040E0F70895DC01CB01FC0156
:105F1000F999FECF06C0F2BDE1BDF89A319600B402
:105F20000D9241505040B8F70895F999FECF92BDB7
:105F300081BDF89A992780B50895A8E1B0E042E0C4
:105F400050E0E5CFDC01A40FB51F4150504040F0B8
:105F5000CB01840F951F2E9105D041505040D8F7AA
:105F60000895262FF999FECF92BD81BDF89A019729
:105F700000B4021639F01FBA20BD0FB6F894FA9A91
:105F8000F99A0FBE08950396272FECDFEADF252F3D
:105F9000E9DF242FE7CF0196272FE4DFE2CFDC01F2
:105FA000CB0102C02D9105D041505040D8F7089543
:105FB000262FF999FECF1FBA92BD81BD20BD0FB625
:105FC000F894FA9AF99A0FBE01960895F894FFCFC3
:105FD000C90ACE0AD00AD50AE50AE50AE50AE50AA1
:105FE000E50AE50AE50AE50AD70ADB0ADE0AE30A5A
:105FF000F30AF90AFD0A8A10B010B610B010B610F4
:1060000008112911B6102F123C12281C901C301CAC
:10601000FA1BFE1B341C021C381C441C0E1C891C61
:10602000121C481C161C4C1C711C1A1C501C781C81
:10603000201C561C5E1C061C3C1C0A1C401C241CFC
:106040005A1C681C811C871CF41B2C1C971CCA1B27
:10605000D01BBD1BC41BD61BDC1BE21BB21DB21D1B
:106060001F1E1F1EC01EDD1ECC1DCC1DE21E511F9B
:10607000611F611F942BAF2BB62BF229F229E92B5C
:10608000FA2B0D2C4E2C532C7E2C8F2CA42CA72CB1
:10609000E029E429152A212A2C2A372ADE29DE299B
:1060A000DE29DE297F2B3A2A3D2A412A6D2AAA2A97
:0660B000AD2AAF2AE32A2D
:1060B60028081E0AFA09770D8D0D920D970D6E0DA3
:1060C600AF0001500114000001000101F44F419599
:1060D6003AD9D4AA004422B684016201AC008A02ED
:1060E600A302C302F5F4F1333267F7F6F030313428
:1060F60097969495939237E200E900EA00B500B6C8
:1061060000B700CD008301CC008A019201940121E1
:1061160002230224022502260227022A02B300B421
:10612600006F0070009F01CB019F02A002E200E910
:1061360000EA00B500B600B700CD008301CC008AA6
:10614600019201940121022302240225022602273C
:10615600022A02B300B4006F0070009F01CB019FBA
:0461660002A0020091
:00000001FF
